:030000000219FDE5
:03000B000200AA46
:03002B0002015778
:03005B000202E9B5
:030073000202D6B0
:1000800002030406080C10182030406080040608A3
:100090000C10182030406080A0C00003070F1F0D17
:1000A0000D04050D050205030302C2AFC0D0C0E078
:1000B000206214E5256009E473E525F4F58AD2622F
:1000C000D0E0D0D0D2AF3285268AC262E526F46075
:1000D0002AD0E0D0D0C295C294C293D2AF32C2959A
:1000E000C294C293206F0D20660A7405D5E0FDE529
:1000F0007BF45290D0E0D0D0D2AF32758A00C28D5E
:10010000D26201F401B9306805206602D29501B9C6
:10011000306805206602D29401B930680520660275
:10012000D29301B9D29230680A2066077403D5E0F1
:10013000FDD29501B9D29130680A2066077403D5C3
:10014000E0FDD29401B9D29030680A2066077403AA
:10015000D5E0FDD29301B9C2AFC2AD53E6EFC0D036
:10016000C0E0D2D3D2AFC2CEE52A600720744915D1
:100170002A21B87800790020742EE580307E01F4C1
:1001800030E70278FF53DACF207E0343DA20307E57
:100190000343DA10C2D8C271E580307E01F430E743
:1001A0000279FFC3E89970CB306103752A18207477
:1001B00003752A18885CD27020740DE52B60041535
:1001C0002B21C843DA01C2D82070024137A85C2035
:1001D0006102C2702074367982B70431C3E894F0AA
:1001E000400374F0F8E8C4540F28F87984B7030288
:1001F000410DC313C3138721200802C313200A062D
:10020000C3C898F8410D28F8500374FFF88822E518
:100210002D54066022206B1FE536C333C333F8E547
:1002200064C313C313F9C3952240028922E825222F
:10023000F52250037522FF7882B6044E852224A849
:1002400024C3E52495614002A861C3E89563400298
:10025000A8638825E56670024188C3E8AA669A50BB
:1002600003E8FAE4F9EAC333FBE568F45B29400DDF
:100270002567F8E56760021567400B41880AC3E50A
:10028000679A5002056778FF8826C3E525944040A9
:1002900002D26420CF0AD0E0D0D043E610D2AD32F3
:1002A000C2CF053A7801E52A6005307402152AC3E9
:1002B000E55C94014005755F0041CC75600075698F
:1002C00000E55F2401F55F5003755FFFD0E0D0D0FB
:1002D00043E610D2AD32C2AF53E67F7592FA759302
:1002E000FFC260759104D2AF32C2AF53E6EFC2AD28
:1002F000C0D0C0E0C0F0D2D3D2AFA8FBA9FCC2D816
:10030000307102615053DACF207E0343DA10307E21
:100310000343DA20D271E580307E01F420E70261E8
:100320002788278928A17D53DACF207E0343DA204E
:10033000307E0343DA10C2D8C271307402A16978EA
:1003400000E580307E01F430E702A169885CA151AC
:1003500053DACF207E0343DA20307E0343DA10C223
:1003600071206102812953DACF207E0343DA1030F5
:100370007E0343DA20C2D8D27188578958C3E895E2
:1003800055F8E99556F97B007E087A00C3E8948C0D
:10039000E994005005755B00811B882178A2E6A8CE
:1003A000216055C3E894C8E994005008E4D2E4FB06
:1003B0007A0A61F6C3E89468E994015008E4D2E34C
:1003C000FB7A0F61F6C3E894D0E994025008E4D2B6
:1003D000E2FB7A1E61F6C3E894A0E994055008E4B4
:1003E000D2E1FB7A3C61F6C3E89498E9940850089E
:1003F000E4D2E0FB7A787E00C3E89559FCE9955A8F
:10040000FD30E70AECF42401FCEDF43400FD755BEB
:1004100000C3EC9AED9E5003755B018859895A859B
:1004200057558558567802A151C3E89527F8E995A4
:1004300028F9307C02A135307B02A135307A02A147
:100440002E207502814CE9FDE8FC816BE9C313F9AC
:10045000E813F8307902A12EE9C313F9E813F83054
:100460007802A12EE9C313FDE813FC20612CC3EC34
:0E047000941CED940240028182ED701EC3ECDC
:10047E0094C850180529E52970021529C3E5299459
:10048E000A5002A169755C00D270A169E52960026B
:10049E0015297888E6F97400207F087896B903024A
:1004AE00789EE624FAFEE43400FFC3EC9EFCED9F3A
:1004BE00FD9208B90310A2085007207609D2768162
:1004CE00D4307602C276A2085016B9030DECF4248D
:1004DE0001FCEDF43400FD0204EE78007900A13544
:1004EE00B90315EC33FCED33FDC3EC940AFCED942B
:1004FE0000FD50047C007D00C3EC94FFED940040A1
:10050E000678FF7900A135EC8572F0A4C5F0A2F74C
:10051E0033F87900400302055178FF790002055146
:10052E00E9C313F9E813F8307C0EE9600278FFC3D3
:10053E00E81338F8E43400F9C3E894FFE994004076
:10054E000278FF885CD270206102A169741FF45595
:10055E002F4BF52FC274EB7002D274752A183074BB
:10056E0003752A0A306102A17D20740353DAFE203E
:10057E007403752B06D0F0D0E0D0D0D2AD43E61088
:10058E003279010205AD79030205AD790A0205AD96
:10059E00791E0205AD79640205AD79C80205AD7804
:1005AE0017E4D5E0FDD8FAD9F6227A147B78020545
:1005BE00D47A107B8C0205D47A0D7BB40205D47AE2
:1005CE000B7BC80205D47902E4D291D5E0FDD2941A
:1005DE00D5E0FDC294D5E0FDC291D5E0FDE920E065
:1005EE0002D29530E002D293E573D5E0FDE920E02A
:1005FE0002C29530E002C2937496D5E0FDD9C9EAE5
:10060E00F8D5E0FDD8FBDBBED29122C37C007D0085
:10061E0075F00005F0EA33FAEB33FB50F6EB13FB03
:10062E00EA13FAC3E9FFE8FEE89AF8E99BF95004E9
:10063E00EFF9EEF8B3EC33FCED33FDD5F0DFEDF969
:10064E00ECF822E889F08A20D2D4F8A9F07B0030A9
:10065E00F70B7BFFF42401F8E9F43400F9E8852068
:10066E00F0A4ADF0F8E98520F0A4AFF0FEED2EF980
:10067E0074003FFA7C04C3EA13FAE913F9E813F89D
:10068E00DCF48BF030F70AE8F42401F8E9F43400D6
:10069E00F9E889F0C2D4F8A9F0227882B6040302F0
:1006AE000703C3E55C940140030206CD852224E4D2
:1006BE00F544F545F546F547F548C26E0207037851
:1006CE0082E6FCD26EE522F523783879C7AA40ABD4
:1006DE0041C3EB13FBEA13FAEC146013C3EB13FBE9
:1006EE00EA13FAEC14146007C3EB13FBEA13FAD106
:1006FE00198844894522C3E5449523F8E5459400BD
:10070E00F9500CC3E89480E994FF4016020734C3F5
:10071E00E8947FE994005003020734787F79000251
:10072E000734788079FF8849894A22E5492546F8B9
:10073E00E54A3547F9854A20E4300701F43548FA91
:10074E0030E709C3EA94F04015020772C3EA940F2A
:10075E00500302077278FF79FF7A0F020772780052
:10076E0079007AF0C3E5249561500AC3740195248B
:10077E00500B020790E54A20E70E020790E54A303B
:10078E00E706884689478A482278A5E6FAC3E549EE
:10079E0033F8E54A33F9D151E930E70BC3E89480D9
:1007AE00E994FF4013E1CAC3E8947FE99400500234
:1007BE00E1CA787F7900E1CA788079FFE820E715F1
:1007CE00C3E52398F84009C3E8940140030207F1FA
:1007DE0078010207F1E8F424012523F8400302070B
:1007EE00F178FF884B2278A6E6FAA847A948D1519E
:1007FE00E930E70CC3E89401E994FF40160208259E
:10080E00C3E894FFE99400500302082578FF7900AD
:10081E00020825780179FFE920E715C3E54B98F822
:10082E004009C3E89401400302084C780102084CC9
:10083E00E8F42401254BF8400302084C78FF882485
:10084E002278FFC26420693D206A12D264C3E5415A
:10085E00940A4009C3E52594405002C26479A1E789
:0F086E006023E541601F74FF8541F0848539F0F8
:10087D00306A0375F005A4F8C5F0600278FFC3E88F
:10088D0095645002A864886322C3E5409440E54115
:10089D009401E56350031401A7046002F56322027D
:1008AD0008AF2275E890227883E6FFE5E820ECF7A3
:1008BD00A8BDA9BE0570C3E57094084052757000BF
:1008CD00E9FA79A0E76044EA7007E571601B020858
:1008DD00EAC3E895716010E5715006600C140208CA
:1008ED00F60460F90208F6E571F571C3946D401BCD
:1008FD007561C0C394044013756180C39404400BAB
:10090D00756140C39404400375610075BB0622E513
:10091D00612410500274FFF5617982B704022143FE
:10092D00C3A861E524985002A824C3E8956340024A
:10093D00A86388258826E570B4070375BB1022745B
:10094D003279A787F0A4C5F0A2F733F8C3E8956113
:10095D004002A8618822882488258826886422750B
:10096D0040007541F022C2AF75C820A8CCA9CDAA10
:10097D003A30CF010A75C824D2AFAB3BAC3C883BB3
:10098D00893CC3E89BF8E99C206908F9306702416E
:10099D007F21DCAD3D8A3DF9EA9DFA600478FF794F
:1009AD00FFAE3EAF3F8B3E8C3FA83BA93CC3E89EBC
:1009BD00F8E99FF9C3E54113FBE54013FAE82AF581
:1009CD0040E93BF54150067540FF7541FF4126AAB0
:1009DD0040AB41AC40AD417E047F02C3EB9404407B
:1009ED00021E1FC3EB940840021E1FC3ED13FDEC46
:1009FD0013FCDEF7C3EA9CFAEB9DFBEF6009C3E93C
:100A0D0013F9E813F8DFF7EA28FAEB39FB8A408B84
:100A1D004150067BFF8B408B41C3EB94025002D2B9
:100A2D00673069047F0341517892E6FFC3E537943F
:100A3D008240110FC3E53794A040010FC3EF940618
:100A4D0040027F057E02E541C4540FF9E541C454CF
:100A5D00F0F8E540C4540F28F8C3E89EFAE9940075
:100A6D00FB4009C3EA9402EB940050047A02E4FBC4
:100A7D0041CBAA40AB41EBC4FEEAC4540F4EFCC3BC
:100A8D00EA9CFAEB9400FBC3E813C313F8EA28FAC7
:100A9D00EB3400FB8A408B41C3EB94024002C267EA
:100AAD007802EBC4FE7B00EAC4540F4EFAC3EA98F9
:100ABD00FA4005C3940250027A027892E6FF306044
:100ACD000241CB855192855293D26043E680C3E4B7
:100ADD009AF8E49BF93067026157E8FAE9FBD3E92C
:100AED0013FDE813FC88518952C3EF94036038EF6E
:100AFD0020E00DE82CF8E93DF9ECFAEDFB020B20B6
:100B0D00E828F8E939F9C3E82402F8E93400F97A5C
:100B1D00FE7BFFC3EF9403400E8A538B54884D899F
:100B2D004E8C4F8D50618B885389548A4D8B4E8CD2
:100B3D004F8D503069127553F07554FF754FF07528
:100B4D0050FF7551F07552FF618BE8FAD3E813FC35
:100B5D008851C3EF94036020EF20E007E82CF8ECF8
:100B6D00FA6177E8282402F87AFEC3EF940340086F
:100B7D008A53884D8C4F618B88538A4D8C4FE56815
:100B8D00C3335002646BF5683060026195753402B1
:100B9D00D26043E680E52D54066034A840A941C3D8
:100BAD00E913F9E813F8C3E913F9E813F830690408
:100BBD00E92440F9C2AF53E67F759100C3E498F57F
:100BCD0094E499F595759104D26043E680D2AF22F5
:100BDD00D265754300752000306C03752040020B03
:100BED00FCD265754300752040306C03752000788C
:100BFD00017901206720E52D54066002C265791444
:100C0D00E541C313700104F8C39414400278143005
:100C1D006904781B791B206010E543600C30690373
:100C2D00D53404D26D819E719D0543E59B5440B52D
:100C3D002002818830690908C3E899400118812391
:100C4D0020650A08C3E899400261FC8123C265C290
:100C5D00AF53E67F7591003067127594007595FE60
:0E0C6D00759104D26043E680D2AF61FCAE40C8
:100C7B00AF41C3E49EF594E49FF595816DC3E533D5
:100C8B009401500261FC30650261FCD802819C81A9
:100C9B0023C26DC2AF53E67F759100855394855483
:100CAB0095759104854D92854E93D26043E680D223
:100CBB00AFE52D54066008206A020533020CDA30CA
:100CCB006D0D206C0A2065071581158102155D22BB
:100CDB0078003064053065027801E53775F007A4BC
:100CEB00F9E5F028F5F0E9A2F013A2F113A2F21343
:100CFB00F537C394785003753778C3E5379538408B
:100D0B0008D266C295C294C293306002A114854F7B
:100D1B0092855093D26043E68022207D16C2AF7538
:100D2B004202D291C292306202D293D2AF759F111E
:100D3B00020F14C2AF754202D291C290306202D23E
:100D4B0095D2AF759F11020F14307243207D20C2D4
:100D5B00AF754203900135757B02C293D29030621E
:100D6B0004D294A172C291D2AF759F01020F14C22B
:100D7B00AF754203900135757B02C295D2923062FA
:100D8B0004D294A192C291D2AF759F21020F14206D
:100D9B007D17C2AF754203900110C293306202D22D
:100DAB0094D2AF759F01020F14C2AF75420390012D
:100DBB0010C295306202D294D2AF759F21020F14EC
:100DCB00207D16C2AF754204D292C290306202D21D
:100DDB0094D2AF759F21020F14C2AF754204D2900B
:100DEB00C292306202D294D2AF759F01020F1430BF
:100DFB007243207D20C2AF754205900124757B04A0
:100E0B00C294D291306204D295C118C292D2AF75FE
:100E1B009F11020F14C2AF754205900146757B01FD
:100E2B00C294D291306204D293C138C290D2AF75C2
:100E3B009F11020F14207D17C2AF7542059001065A
:100E4B00C294306202D295D2AF759F11020F14C2B9
:100E5B00AF75420590011AC2943062EBD293D2AFB8
:100E6B00759F11020F14207D16C2AF754206D290EA
:100E7B00C291306202D295D2AF759F01020F14C29C
:100E8B00AF754206D292C291306202D293D2AF7545
:100E9B009F21020F14307243207D20C2AF75420197
:100EAB00900146757B01C295D292306204D293C1F8
:100EBB00BEC290D2AF759F21020F14C2AF75420113
:100ECB00900124757B04C293D290306204D295C1F9
:100EDB00DEC292D2AF759F01020F14207D17C2AFF5
:100EEB0075420190011AC295306202D293D2AF754E
:100EFB009F21020F14C2AF754201900106C29330BD
:100F0B006202D295D2AF759F01C266229001047521
:100F1B007B00C295C294C293D292D291D290C262FC
:100F2B0022788076090876090876040876FF087619
:100F3B00030876FF08760A08760108760108760121
:100F4B00788C76010876FF0876FF0876FF0876FF27
:100F5B000876FF0876030876FF0876FF0876FF0809
:100F6B0076250876D0087628087650087604087619
:100F7B00FF08760208760008767A0876FF08760175
:100F8B00087601087600087603087600227887E653
:100F9B00FFC2727888E6C394036008C27DE630E135
:100FAB0002D27DC27E7889E630E102D27EC3EF9415
:100FBB00026008758E01D273020FCB758E00C2735F
:100FCB00227880E6149000809378A5F67881E61459
:100FDB009000809378A6F67886E61490008D93782F
:100FEB00A7F67886E6F539C3940250037539027873
:100FFB009CE67538FFB402037538A0B4030375384B
:10100B008278A3E61490009A93F566120F172222AA
:10101B007896E6FA7897E6FB7888E6B40305C3EB97
:10102B00940EFB307F047A007BFFC3EB9AFCC394D6
:10103B008250027C827572000572EC8572F0A4C33B
:10104B00E5F0947D40F222D27F111B12059E7A00AF
:10105B007B007C10120594E55C2AFA74003BFBDCE8
:0F106B00F37C04C3EB13FBEA13FADCF7FEC27F3E
:10107A00111B22E5EF20E6037520000520903FFFB3
:10108A00E520146006901DFF146000930460037548
:10109A00EF1253D9BF7581C043FF8012058F75EFD8
:1010AA000243B203E5B3240220E70DF521E5E3206C
:1010BA00E0068521B343E301120F177580FF75A47B
:1010CA000075F19075D47F75908775A5BF75F2BFCD
:1010DA0075D50075A60175E241120F17E4F8F6D826
:1010EA00FD756801120F2C1215AE7898867375304B
:1010FA0001C2AF1205A81205B812059E1205BF1249
:10110A00059E1205C612059EC2AF78FA79FA308793
:10111A0007D9FBD8F7021C00120F98120FCC111A2C
:10112A00111B78988673120F1775881075890275C6
:10113A00C82475910475D84075A82275B80275E659
:10114A0090759B80759D0075D10E75BC5875BB0650
:10115A0075BA1175E88012058FD2AF1208AC7536D0
:10116A000053DACF207E0343DA20307E0343DA10BD
:10117A0043DA01C2D8C2711205A8D2617B037A0C84
:10118A00E55B70077A0CDB0302111212059E2070D0
:10119A0003021112C270E55CC3940240E1E52F54C8
:1011AA001F855E5DF55EB55DD5DAD5C26153DACFCE
:1011BA00207E0343DA20307E0343DA10C2D8C2719C
:1011CA0078A2E67008D274E52F54E0F52FC275753F
:1011DA0029001205A3307409C3E529940A4002D2F2
:1011EA007512059478023074027800C3E55C984061
:1011FA00F0C2AF1205B81205B81205B8D2AF12057F
:10120A00A8754C007888E6B4030241EA120594787E
:10121A008CE6C3940150030212EAE530C3940150EC
:10122A00030212EA207435C3E55C94FF50030212EC
:10123A00EAC2AF1205CDD2AF1205A3C3E55C940191
:10124A0050EFC2AF1205B81205991205B8D2AF1203
:10125A0005A3C3E55C94FF40E90217567F02D27FDB
:10126A00111B1205A3C2AFC27F111BAE5CC3E55CA2
:10127A00947FD2AF407412058FC2AF1205CDD2AFA0
:10128A00DFDC1152C3EE7897F61205A81215F01298
:10129A0016D97F0AD27F111B1205A3C2AFC27F11D2
:1012AA001BAE5CC3E55C947FD2AF50E612058FC2D9
:1012BA00AF1205B81205991205B8D2AFDFD611528E
:1012CA00EE24037896F61205A81215F012170812E2
:1012DA0005A3111BC3E55C94FF5002412E02175669
:1012EA00C3E55C954C4003855C4C1205A3780179F3
:1012FA0088E7B403027805C3E55C984002410EC250
:10130A00AF1205CD1205CD1205CDD2AF1205A875C3
:10131A003000E4F531F5320531E531F4703F05323C
:10132A00789AE67819146012783214600D787D1470
:10133A00600878FA146003753200C3E53298401DDC
:10134A00120F1712058F153275310078998673C2FC
:10135A00AF1205CDD2AF789886731205A3120599FC
:10136A00E52A700530740221127801207402780689
:10137A00C3E55C9840A17888E6C39403600312052C
:10138A00A3E52A7003021112C2AF120F17E4F52265
:10139A00F523F524F525F526F567D2AF7885E6C35A
:1013AA0033F565E4F544F545F546F547F548F57036
:1013BA00F52CF52DF53775700875BB1012058F12CF
:1013CA0008B0E5E820ECFBA8BDA9BEE97001F888E1
:1013DA00711208B475700875BB10120F98C2AF75F8
:1013EA0061FF12094C852261852262852263D2AF90
:1013FA0075220175240175250175260185606975B7
:10140A006A017888E6B40307C27D307602D27DD2BB
:10141A0068D269753300120E71120EA012096C128D
:10142A00097312096C12097312096C120BEE120677
:10143A00A8120CDB120D25120973120BDD306E0394
:10144A0012070420670312084F3067031208961226
:10145A000CDB120D54120973120BEE306E031207D5
:0D146A0039120CDB120DCB120973120BDDD1
:10147700306E03120797120CDB120DFA1209731262
:101487000BEE306E031207F4120CDB120E71120909
:10149700731208B0120BDD120CDB120EA01208B487
:1014A7001209733069328564618564628560697584
:1014B7006A0179187A0CC3E53399400FC269D26A79
:1014C7008A358564618564630214DFC3E55C940132
:1014D7004003021435021565306A1D206C1AE53584
:1014E700147006C26AD26B8135F535C3E55C940189
:1014F700400302143502156575360078FA79A4E7BA
:1015070060027803C3E55F985054307404E52A609D
:101517004D7888E6B40317207D05207607A135307E
:101527007602A135206C07D26C856461817478F0EE
:10153700306C058564617820C3E541985002813598
:10154700306C1BC26CC27D307602D27DD26A753593
:101557001285646181350536E55C6002A1687536E0
:1015670000C2AF120F177887E6FE7602120F98783F
:1015770087EEF6E4F522F523F524F525F526F5653E
:10158700752C00752D00D2AF1205A3120F1778A482
:10159700E66006C292C291C290307409C3E53694E0
:1015A7000440022112611C901A0D7820121632E5B0
:1015B70020B4550CA3121632E520B4AA030215D0A5
:1015C700120F2C1215F00215EF901A0378807B0A80
:1015D700121632A308DBF9901A0F788C7B191216B2
:1015E70032A308DBF9901A2822C2AF12167112161D
:1015F7004B901A00740E121637A37406121637A3EF
:101607007415121637901A0378807B0A121636A3C0
:1016170008DBF9901A0F788C7B19121636A308DBB2
:10162700F9121684121662901A2822E493F622E61B
:10163700438F01538FFD75EF0275B7A575B7F1F0AD
:10164700538FFE22438F02438F0175EF0275B7A5B3
:1016570075B7F1901A0DF0538FFC22901A0D74553F
:10166700D137901A0E74AAD137227A3079D07820E0
:10167700901A40D132E520F709A3DAF7227A3079B8
:10168700D0901A40E7D13709A3DAF922AB74A875CD
:10169700BB01027980BB02027981BB03027982BB5D
:1016A70004027984BB05027986BB06027992BB07DF
:1016B700027987BB080279A3BB0902799CBB0A029E
:1016C7007988BB0B027989E8F7227C051205A8DC2B
:1016D700FB22C2AF1205B81205BF1205C61205CD0F
:1016E7001205991205B81205BF1205C61205CD12CB
:1016F70005991205B81205BF1205C61205CDD2AF5E
:1017070022C2AF1205CD1205C61205BF1205B812C7
:1017170005991205CD1205C61205BF1205B81205A7
:10172700991205CD1205C61205BF1205B8D2AF2210
:10173700AE74AF75C2AF1205B81205B81205B8126C
:101747000599DEF21205CD120599DFF8D2AF22D145
:10175700D9D1D1D1D1757401757501757600F1377D
:101767007C05AD5C1205A8C3ED955C70F5C3E55C1F
:101777009401400AC3E55C94FF4032021792D1936B
:10178700B1F0D1D9C2AF75EF12D1D1DCD50576C38F
:10179700E5769403500280C6D1D10575E57414909F
:1017A700009F93F808C3E57598500280AED1D1D158
:1017B700D10574C3E574940C5002809C120F2CB1B0
:0817C700F0C2AF75EF12D1D1A1
:0319FD0002107D58
:101A00000E0615090904FF03FF0A01010155AA0189
:101A1000FFFFFFFFFF03FFFFFF25D0285004FF0259
:091A2000007AFF0101000300FF40
:101A400023585031384123202020202020202020DE
:101A500023424C48454C4923463333302320202031
:101A60002020202020202020202020202020202076
:101C0000C2AFC2D353D9BF7581C043B20343FF8073
:101C1000752438752503B1C975EF0275E24043F1AB
:101C20008053A47F75D4FFD2877DFA780379E67C50
:101C300010752200752300901DD67B0675249875BB
:101C400025013087028142208708D8FBD9F9DCF7CB
:101C500081B4308708D8FBD9F9DCF781B4B189E4C5
:101C600093A3C39A6004DDC381B4DBDBB17B600264
:101C7000812B7B08E493FAA3B15CDBF87A30B15C8A
:101C8000752200752300B17BEAFCEBFDC3ED94FEE9
:101C9000400EB17B8A278B28ED30E0048A828B834B
:101CA000B17B7AC270D8C3ED94FE601350CEBD00F4
:101CB00025EC60097520007521FF0200008100A855
:101CC00027A9280809D804D90281D3B17FEA89AAB3
:101CD000F281C50D81A0C3ED94035049EDA2E092BD
:101CE000007AC5C3E5829400E583941C50902000DF
:101CF00010438F02438F0175B7A575B7F1F030001F
:101D00001FA827A9280809438F01538FFDD804D99C
:101D100002A12089AAE275B7A575B7F1F0A3A10DBC
:101D2000538FFC817C7AC1BD030CE493A3FAB140CC
:101D3000DCF8B138817C817EAA22AB23B15CEBFA5E
:101D4000EA6222752608C3E52313F523E52213F57D
:101D50002250066323A0632201D526EAB1C9B1C986
:101D600075260AEAF4200102D287300102C287B147
:101D7000C9C3134002C201D526EB22B17FEAFB2082
:101D80008702A17F308702A184752608AE24AF2583
:101D9000C3EF13FFEE13FEB1CDB1C9C3EA13308711
:101DA000024480FA30E703632201C3E52313F523DD
:101DB000E52213F52250066323A0632201D526D91C
:101DC000E52265236523F52222AE24AF250E0FDE22
:101DD000FEDFFCD20122424C48656C693437316326
:041DE000F3300601D5
:00000001FF
